:100000000C945E000C9486000C9486000C94860080
:100010000C9486000C9486000C9486000C94860048
:100020000C9486000C9486000C9486000C94860038
:100030000C9486000C9486000C9486000C94860028
:100040000C9434020C9486000C94A4020C947E024E
:100050000C9486000C9486000C9486000C94860008
:100060000C9486000C9486000000000024002700F9
:100070002A0000000000250028002B0004040404CE
:100080000404040402020202020203030303030342
:10009000010204081020408001020408102001021F
:1000A00004081020000000080002010000030407FB
:1000B0000000000000000000D602460411241FBE0C
:1000C000CFEFD8E0DEBFCDBF22E0A2E9B1E001C0B2
:1000D0001D92A534B207E1F711E0A0E0B1E0E6E13E
:1000E000FDE002C005900D92A239B107D9F710E0EA
:1000F000CDE5D0E004C02197FE010E948604CC35F6
:10010000D107C9F70E9461030C947E060C9400008D
:10011000EBEAF0E02491E7E9F0E09491E3E8F0E025
:10012000E491EE23C9F0222339F0233001F1A8F441
:10013000213019F1223029F1F0E0EE0FFF1FEE58C7
:10014000FF4FA591B4912FB7F894EC91811126C07F
:1001500090959E239C932FBF08952730A9F02830B7
:10016000C9F0243049F7209180002F7D03C02091F1
:1001700080002F7720938000DFCF24B52F7724BD18
:10018000DBCF24B52F7DFBCF2091B0002F772093BC
:10019000B000D2CF2091B0002F7DF9CF9E2BDACFC7
:1001A0003FB7F89480919A0190919B01A0919C0196
:1001B000B0919D0126B5A89B05C02F3F19F001966F
:1001C000A11DB11D3FBFBA2FA92F982F8827BC01B1
:1001D000CD01620F711D811D911D42E0660F771FD9
:1001E000881F991F4A95D1F708958F929F92AF92D9
:1001F000BF92CF92DF92EF92FF924B015C010E947F
:10020000D0006B017C010E94D0006C197D098E0921
:100210009F09683E734081059105A8F321E0821A89
:100220009108A108B10888EEC80E83E0D81EE11C31
:10023000F11C81149104A104B10429F7FF90EF90FF
:10024000DF90CF90BF90AF909F908F900895AF9226
:10025000BF92CF92DF92EF92FF920F931F93CF93B3
:10026000DF936C017B018B01040F151FEB015E0115
:10027000AE18BF08C017D10759F06991D601ED91AA
:10028000FC910190F081E02DC6010995892B79F749
:10029000C501DF91CF911F910F91FF90EF90DF90FB
:1002A000CF90BF90AF900895FC01538D448D252FC2
:1002B00030E0842F90E0821B930B541710F0CF9600
:1002C000089501970895FC01918D828D981761F032
:1002D000A28DAE0FBF2FB11D5D968C91928D9F5F49
:1002E0009F73928F90E008958FEF9FEF0895FC0128
:1002F000918D828D981731F0828DE80FF11D858DDB
:1003000090E008958FEF9FEF0895FC01918D228D6D
:10031000892F90E0805C9F4F821B91098F739927F2
:1003200008958EE991E00E94850121E0892B09F46E
:1003300020E0822F089580E090E0892B29F00E9430
:10034000910181110C9400000895FC01A48DA80F67
:10035000B92FB11DA35ABF4F2C91848D90E0019607
:100360008F739927848FA689B7892C93A089B18927
:100370008C91837080648C93938D848D981306C0C8
:100380000288F389E02D80818F7D80830895EF922C
:10039000FF920F931F93CF93DF93EC0181E0888F3F
:1003A0009B8D8C8D98131AC0E889F989808185FF0F
:1003B00015C09FB7F894EE89FF896083E889F989B1
:1003C00080818370806480839FBF81E090E0DF91B3
:1003D000CF911F910F91FF90EF900895F62E0B8D06
:1003E00010E00F5F1F4F0F731127E02E8C8D8E11C1
:1003F0000CC00FB607FCFACFE889F989808185FF28
:10040000F5CFCE010E94A501F1CFEB8DEC0FFD2FB2
:10041000F11DE35AFF4FF0829FB7F8940B8FEA89E2
:10042000FB8980818062CFCFCF93DF93EC01888DF1
:100430008823B9F0AA89BB89E889F9898C9185FD5F
:1004400003C0808186FD0DC00FB607FCF7CF8C91ED
:1004500085FFF2CF808185FFEDCFCE010E94A501FF
:10046000E9CFDF91CF9108951F920F920FB60F92AF
:1004700011242F933F938F939F93AF93BF938091BA
:10048000960190919701A0919801B09199013091B6
:10049000950123E0230F2D3758F50196A11DB11DBD
:1004A000209395018093960190939701A0939801D2
:1004B000B093990180919A0190919B01A0919C0128
:1004C000B0919D010196A11DB11D80939A01909359
:1004D0009B01A0939C01B0939D01BF91AF919F910F
:1004E0008F913F912F910F900FBE0F901F901895F5
:1004F00026E8230F0296A11DB11DD2CF1F920F92A5
:100500000FB60F9211242F933F934F935F936F93E6
:100510007F938F939F93AF93BF93EF93FF938EE956
:1005200091E00E94A501FF91EF91BF91AF919F9142
:100530008F917F916F915F914F913F912F910F908C
:100540000FBE0F901F9018951F920F920FB60F922B
:1005500011242F938F939F93EF93FF93E091AE011C
:10056000F091AF018081E091B401F091B50182FD7D
:100570001BC090818091B7018F5F8F732091B8016C
:10058000821741F0E091B701F0E0E256FE4F958FFF
:100590008093B701FF91EF919F918F912F910F90D1
:1005A0000FBE0F901F9018958081F4CF1092A1017B
:1005B0001092A00188EE93E0A0E0B0E08093A20149
:1005C0009093A301A093A401B093A5018AE091E0C8
:1005D00090939F0180939E0185EC90E09093AB01F6
:1005E0008093AA0184EC90E09093AD018093AC01DC
:1005F00080EC90E09093AF018093AE0181EC90E0AD
:100600009093B1018093B00182EC90E09093B3019C
:100610008093B20186EC90E09093B5018093B40191
:100620001092B7011092B8011092B9011092BA015C
:1006300010923C0210923B0210923E0210923D0238
:100640001092400210923F0269E770E090E080E073
:100650000E94B105009701F190933C0280933B0208
:1006600028E730E030933E0220933D0220913F0284
:1006700030914002232B11F4FC01108288E790E0B6
:100680009093400280933F0268E171E080913B02C9
:1006900090913C020C94770680913B0290913C0231
:1006A000009711F00E94280510923C0210923B0224
:1006B0001092400210923F0210923E0210923D02B0
:1006C0000895789484B5826084BD84B5816084BDCA
:1006D00085B5826085BD85B5816085BD80916E00E0
:1006E000816080936E001092810080918100826011
:1006F000809381008091810081608093810080914E
:1007000080008160809380008091B100846080933C
:10071000B1008091B00081608093B00080917A0038
:10072000846080937A0080917A00826080937A005E
:1007300080917A00816080937A0080917A0080684D
:1007400080937A001092C100E091AE01F091AF0168
:1007500082E08083E091AA01F091AB011082E091E8
:10076000AC01F091AD018FEC80831092B601E09165
:10077000B201F091B30186E08083E091B001F09185
:10078000B101808180618083E091B001F091B1017D
:10079000808188608083E091B001F091B101808117
:1007A00080688083E091B001F091B10180818F7DFC
:1007B0008083E7E9F0E02491E3E8F0E08491882386
:1007C00099F090E0880F991FFC01E859FF4FA5911F
:1007D000B491FC01EE58FF4F859194918FB7F89436
:1007E000EC91E22BEC938FBF80E0E82E80E0F82EB6
:1007F00000913F02109140021093940100939301E5
:10080000D0E0C0E0C017D1077CF580913F02909105
:100810004002C817D90720F0109292012196F2CF1A
:1008200080913B0290913C020097B1F38C0F9D1F89
:10083000FC01808180939201803339F462E370E09F
:1008400080E090E00E94F500E9CF813339F781E044
:100850000E94880062E370E080E090E00E94F50072
:1008600080E00E948800DACF68EB7BE080E090E0D7
:100870000E94F500E114F10409F4BACF0E9491013D
:10088000882309F4B5CF0E940000B2CF80913B02CB
:1008900090913C02009711F00C94280508952F9236
:1008A0003F924F925F926F927F928F929F92AF9200
:1008B000BF92CF92DF92EF92FF920F931F93CF934D
:1008C000DF93CDB7DEB7CA1BDB0B0FB6F894DEBFE4
:1008D0000FBECDBF09942A88398848885F846E840A
:1008E0007D848C849B84AA84B984C884DF80EE8054
:1008F000FD800C811B81AA81B981CE0FD11D0FB65D
:10090000F894DEBF0FBECDBFED010895EE0FFF1FBF
:100910000590F491E02D09940F931F93CF93DF93EB
:100920008230910510F482E090E0E0914302F09172
:10093000440230E020E0B0E0A0E0309799F42115C7
:10094000310509F44AC0281B390B24303105D8F58C
:100950008A819B816115710589F1FB0193838283F3
:10096000FE0111C04081518102811381481759074E
:10097000E0F04817590799F4109761F012960C931C
:10098000129713961C933296CF01DF91CF911F914E
:100990000F9108950093430210934402F4CF211560
:1009A000310551F04217530738F0A901DB019A01D4
:1009B000BD01DF01F801C1CFEF01F9CF90934402EF
:1009C00080934302CDCFFE01E20FF31F81939193F9
:1009D0002250310939832883D7CF209141023091A9
:1009E0004202232B41F42091020130910301309304
:1009F0004202209341022091000130910101211512
:100A0000310541F42DB73EB74091040150910501E5
:100A1000241B350BE0914102F0914202E217F307EB
:100A2000A0F42E1B3F0B2817390778F0AC014E5F5E
:100A30005F4F2417350748F04E0F5F1F5093420257
:100A400040934102819391939FCFF0E0E0E09CCFEF
:100A5000CF93DF930097E9F0FC0132971382128263
:100A6000A0914302B0914402ED0130E020E01097E4
:100A7000A1F420813181820F931F20914102309196
:100A800042022817390709F061C0F0934202E0934F
:100A90004102DF91CF910895EA01CE17DF07E8F513
:100AA0004A815B819E0141155105B1F7E901FB8344
:100AB000EA8349915991C40FD51FEC17FD0761F4E2
:100AC000808191810296840F951FE9019983888323
:100AD000828193819B838A83F0E0E0E012968D917E
:100AE0009C9113970097B9F52D913C911197CD01E9
:100AF0000296820F931F20914102309142022817E3
:100B0000390739F6309751F510924402109243029A
:100B1000B0934202A0934102BCCFD383C2834081F1
:100B20005181840F951FC817D90761F44E5F5F4F3D
:100B300088819981480F591F518340838A819B8105
:100B4000938382832115310509F0B0CFF0934402DD
:100B5000E09343029ECFFD01DC01C0CF13821282DD
:100B6000D7CFB0E0A0E0E7EBF5E00C9451048C01A6
:100B7000009751F4CB010E948C048C01C801CDB7C1
:100B8000DEB7E0E10C946D04FC01E60FF71F9C0159
:100B900022503109E217F30708F49DC0D901CD9125
:100BA000DC911197C617D70798F0C530D10530F3FF
:100BB000CE0104978617970708F3C61BD70B229719
:100BC000C193D1936D937C93CF010E942805D6CF1A
:100BD0005B01AC1ABD0A4C018C0E9D1EA091430214
:100BE000B0914402512C412CF12CE12C109731F59D
:100BF00080914102909142028815990509F05CC0EC
:100C00004616570608F058C08091000190910101E6
:100C1000009741F48DB79EB74091040150910501B2
:100C2000841B950BE817F90708F055C0F0934202B2
:100C3000E0934102F90171836083A0CF8D919C9173
:100C4000119712966C90129713967C901397A81593
:100C5000B90559F56C0142E0C40ED11CCA14DB047D
:100C600020F1AC014A195B09DA011296159780F060
:100C70006282738251834083D9016D937C93E11426
:100C8000F10471F0D7011396FC93EE93129776CF8F
:100C900022968C0F9D1FF90191838083F301EFCF82
:100CA000F0934402E093430269CF4816590608F4D2
:100CB0002C017D01D3019ACFCB010E948C047C01D1
:100CC000009749F0AE01B8010E946E06C8010E946B
:100CD0002805870153CF10E000E050CFFB01DC0175
:100CE00002C001900D9241505040D8F70895FB0189
:100CF000DC0101900D920020E1F7089510E0CDE5B0
:100D0000D0E004C0FE010E9486042196CE35D107B2
:060D1000C9F7F894FFCFC3
:100D160000004502800000000000C70127015401C1
:100D260014028501630177013031303030303131C2
:100D360030313031303130303031303030313130A7
:100D46003030313031313031303130303031303097
:100D56003031303031313030303130313030313186
:100D66003031313131303131303130303030313075
:100D76003030313130303031303131303131313065
:100D86003030313130313030303131313030313056
:100D96003031303131303031303131313131303143
:020DA60000004B
:00000001FF
